:020000040000FA
:020000000C28CA
:08000800A0000308A10021087B
:100010008300A00E200E0900831686308100FF2386
:10002000900083128501BD284D3475346C347434CE
:1000300069346D346F346434653433342E34303481
:10004000303420340330B000FF30AF0000343230A1
:10005000AA00AA30AB00051EAF010000AB0B2B2895
:10006000851DAE01B70B3928FA30B700B80B392817
:10007000B901AA0B292800343A1C44280000F930A1
:100080006500F93085000034FD306500F9308500E9
:100090000034FF306500FF30850000343A1C5728DB
:1000A0000000F9306500F930850004302828FD3063
:1000B0006500F9308500043028283A1C66280000C5
:1000C000FB306500F930850004302828FD306500DC
:1000D0000430AA006D30AB00FB30051DF9308500FF
:1000E000051EAF01AB0B6C28851DAE01FB30051D55
:1000F000F9308500AA0B6A280034AD010430A8004D
:100100003E188F2822201230BC0004302820B00B6B
:100110008C282F18B7282220BC0B8528932848301C
:100120002820FF30B0002D08B820AC00AC09093001
:10013000A9009D28AC0C031C9F285D20A1284E20FF
:100140000000B00BA6282F18B7282220A90B9A2848
:100150004E20B00BAE282F18B72822204E20B00B0F
:10016000B4282F18B7282220AD0AA80B93280034F2
:10017000820753344334453445348230620064305E
:100180002820FF3065000130B100C8302820FF3042
:10019000B700B800B900B5000A30BC0064302820B0
:1001A00049208519E228643028203C20BC0BCE2849
:1001B0004920851DD928B10A05303102031CE228E7
:1001C0000130B100FF30AE001E30A70027202E1CEA
:1001D000C528A70BE628FF30BA001930BB00143041
:1001E000BC000519F628BC0BF12805291430BC0009
:1001F000051DFD28BC0BF8280529BB0BEF28BA010B
:10020000F9308500FD3065000929F9308500F930A5
:100210006500FF30AE000730A7000518F22927203F
:100220002E1CC528A70B0F293108BF00BF030319D7
:100230002D29BF0303193129BF0303192729BF0340
:1002400003192229FF306500851DC5282429FF30A8
:10025000BE007D202E1CC52829293A1C3529B50150
:1002600051293A185129B10A14292230B2003A29E9
:100270001830B2003C20851DC52805183B29FF30E9
:10028000BE007D202E1CC52805183829B20B412937
:100290003C20BE017D203C202E1CC5280518382995
:1002A0004A29FF30BE007D202E1CC528051E51297D
:1002B000FF30B400B600B9006430B800FA30B700BF
:1002C000851DC52805185129051E9C29602949202E
:1002D000FF30B300C830BC000E3028202E1CC528CB
:1002E0000518E829051E7829BC0B6C29B3016A2979
:1002F0003C20341CAC290D30BD000A3028202E1CB7
:10030000C5280518E829051A9929BD0B7D29B401CE
:100310003318AC293618D1291930BD000A302820ED
:100320002E1CC5280518E829051A6729BD0B8E293A
:10033000D1294920B6016C293C204B30BC000A3041
:1003400028202E1CC5280518E829051AAA29BC0B47
:100350009F29AC29B40167293C200630A700193039
:10036000BC000A3028202E1CC5280518E829051ACB
:100370006729BC0BB129A70BAF29B4013C200B3076
:10038000A7001930BC000A3028202E1CC5280518EB
:10039000E829051A6729BC0BC329A70BC12903301B
:1003A000D4290430D4291830B200B401351CDA291C
:1003B000391CAC292E1CC5280518E829051AE32983
:1003C0007D20B20BDA294430B800FA30B700AC29EE
:1003D0003C20FF302820FF30B900851DC5280518B6
:0803E000ED29D3297D20F2294B
:02400E00D43F9D
:084200000000010002000300B0
:00000001FF
